S01900006F70656E626C745F73746D3332663734362E73726563F8
S3150800000020140020795D0008AD5D0008B15D000888
S31508000010B55D0008B95D0008BD5D00080000000078
S31508000020000000000000000000000000C15D00089C
S31508000030C55D000800000000C95D0008BD10000885
S31508000040CD5D0008D15D0008D55D0008D95D0008C2
S31508000050DD5D0008E15D0008E55D0008E95D000872
S31508000060ED5D0008F15D0008F55D0008F95D000822
S31508000070FD5D0008015E0008055E0008095E0008CF
S315080000800D5E0008115E0008155E0008195E00087E
S315080000901D5E0008215E0008255E0008295E00082E
S315080000A02D5E0008315E0008355E0008395E0008DE
S315080000B03D5E0008415E0008455E0008495E00088E
S315080000C04D5E0008515E0008555E0008595E00083E
S315080000D05D5E0008615E0008655E0008695E0008EE
S315080000E06D5E0008715E0008755E0008795E00089E
S315080000F07D5E0008815E0008855E0008895E00084E
S315080001008D5E0008915E0008955E0008995E0008FD
S315080001109D5E0008A15E0008A55E0008A95E0008AD
S31508000120AD5E0008B15E0008B55E0008B95E00085D
S31508000130BD5E0008C15E0008C55E0008C95E00080D
S31508000140CD5E0008D15E0008D55E0008D95E0008BD
S31508000150DD5E0008E15E0008E55E0008E95E00086D
S31508000160ED5E0008F15E0008F55E0008F95E00081D
S31508000170FD5E0008015F0008055F0008000000003A
S31508000180095F00080D5F0008115F0008155F000889
S31508000190195F00081D5F0008215F0008255F000839
S315080001A0295F00082D5F0008315F0008355F0008E9
S315080001B0395F00083D5F0008415F0008455F000899
S315080001C0495F00084D5F00080EB418B5040008988A
S315080001D0012817D1A06B30F48030A063E168DFF8FE
S315080001E078080140E160E06830F44010E0600F985C
S315080001F0012803D1E06850F48010E060200000F088
S31508000200F0FE0AE0E06850F04000E060200000F0F0
S31508000210E8FEA16B51F48031A1630699012907D143
S31508000220A16851F00601A160A16851F02001A16002
S31508000230C0B212BC5DF810FB1300DBB2022B52D120
S31508000240DFF818288A1ADFF818389A4201D20F21DF
S315080002504FE0DFF810288A1ADFF80C389A4201D2E4
S315080002600E2146E0DFF804288A1ADFF804389A4295
S3150800027001D20D213DE0DFF8FC278A1ADFF8F837AE
S315080002809A4201D20C2134E0DFF8F0278A1ADFF807
S31508000290F0379A4201D20B212BE0DFF8E8278A1AB9
S315080002A0DFF8E4379A4201D20A2122E0DFF8DC2798
S315080002B08A1ADFF8DC379A4201D2092119E0DFF8F9
S315080002C0D4278A1ADFF8D0379A4201D2082110E0DB
S315080002D0DFF8C827891ADFF8C827914201D2072113
S315080002E007E0062105E0D2B2002A01D1092100E083
S315080002F00921C26832F47052C260C268890211F4D8
S3150800030070511143C16000207047816851F00101A6
S315080003108160002070478168490849008160002093
S31508000320704780B5C26832F0C042C2600A00D2B2D5
S31508000330012A08D1C16851F00051C160322000F08D
S3150800034077FE002002BDC9B2002904D1C16851F068
S315080003508041C160F2E70120F4E70EB478B50400E5
S3150800036000252600002005E0002104EB8002C2F8E3
S315080003700411401C0F28F7D30F9800280CD1A06B46
S3150800038030F40010A063206850F040002060206818
S3150800039050F08000206003E0A06B50F40010A063CA
S315080003A0002016F56061086016F50060006816F50D
S315080003B0006108600A9801280CD10798002804D122
S315080003C00021200000F0F7F818E00121200000F0D5
S315080003D0F2F813E00A9803280CD10798002804D1EC
S315080003E00021200000F0E7F808E00121200000F0D5
S315080003F0E2F803E00321200000F0DDF810212000D8
S3150800040000F0B9F8002800D00125200000F0C4F853
S31508000410002800D00125002016F50061086100209B
S3150800042016F500614861002016F50061C8610020D4
S315080004301BE0002116EB401212F51062116006E06F
S315080004405FF0904116EB401212F51062116016EB40
S31508000450401111F5106100220A6116EB401111F5E1
S3150800046010614FF67F328A60401C0599884210D287
S3150800047016EB401111F5106109680029D9D5002835
S31508000480DED15FF0006116EB401212F510621160C2
S31508000490DDE700201BE0002116EB401212F5306262
S315080004A0116006E05FF0904116EB401212F53062DB
S315080004B0116016EB401111F5306100220A6116EB46
S315080004C0401111F530614FF67F328A60401C05995C
S315080004D0884210D216EB401111F5306109680029DF
S315080004E0D9D50028DED15FF0006116EB401212F56F
S315080004F030621160DDE716F50060006930F480703F
S3150800050016F500610861089801280ED1DFF8040B7A
S3150800051016F50061086316F50060006B40F480303C
S3150800052050F0030016F5006630630020A0617FF0E6
S31508000530804060610898002803D1A06950F0100037
S31508000540A061A169DFF8D00A0143A1610B980028D0
S3150800055003D0A06950F00800A0610F98012805D1C2
S31508000560A06940F0804050F00400A0612800C0B2A5
S3150800057072BC5DF810FB0022890151F0200101616F
S31508000580521CDFF8981A8A4204D201698906F7D400
S31508000590002070470320FCE7002110220261491C55
S315080005A0DFF8782A914204D20269D206F7D40020ED
S315080005B070470320FCE710F500621268C9B21143C0
S315080005C010F5006001600020704710F50060806833
S315080005D010F00600002801D1002006E0022801D00C
S315080005E0062801D1022000E00020C0B2704730B4CE
S315080005F00A784B78012B2BD110F50063DB690124AF
S315080006000D7815F00F05AC40A4B2234310F500642D
S31508000610E36110EB421313F510631B681B0440D407
S3150800062010EB421313F510631B688C686405640DA0
S31508000630C97854EA814454EA825444F0805454F404
S315080006400044234310EB421010F51060036028E0C5
S3150800065010F50063DB6901240D7815F00F05AC4031
S3150800066053EA044310F50064E36110EB421313F5F3
S3150800067030631B681B0414D410EB421313F5306364
S315080006801B688C686405640DC97854EA814444F093
S31508000690805454F40044234310EB421010F53060A4
S315080006A00360002030BC704730B40A784B78012BC1
S315080006B028D1012310F50064E46B0D7815F00F05B9
S315080006C013FA05F5ADB2AC4310F50065EC6310F509
S315080006D00064E469097811F00F018B409BB234EA93
S315080006E0030310F50061CB6110EB421111F510619F
S315080006F00B68DFF82C190B4010EB421010F5106050
S31508000700036026E0012310F50064E46B0D7815F00C
S315080007100F0513FA05F534EA054410F50065EC6390
S3150800072010F50064E469097811F00F018B4034EA8A
S31508000730034410F50061CC6110EB421111F53061EC
S315080007400B68DFF8E0180B4010EB421010F530602C
S315080007500360002030BC7047F8B504000D784B786C
S31508000760012B40F0DD804B69002B24D114EB451397
S3150800077013F5106314EB451616F5106636696FF314
S31508000780DC461E6114EB451313F5106314EB45168E
S3150800079016F51066366956F400261E6114EB4513E5
S315080007A013F5106314EB451616F510663669F60C44
S315080007B0F6041E615AE014EB451313F5106314EBA7
S315080007C0451616F510663669F60CF6041E6114EB26
S315080007D0451313F5106314EB451616F510663669BE
S315080007E06FF3DC461E6114EB451616F5106614EB1E
S315080007F0451313F510631F69D1F814C08B6813EB02
S315080008000C0CBCF1010C8B68BCFBF3F3DFF818C8C1
S315080008101CEAC34C5CEA0707376114EB451313F56A
S31508000820106314EB451616F5106636694F697F0393
S315080008307F0B3E431E61CB78012B17D114EB451372
S3150800084013F5106314EB451616F51066366936F07F
S31508000850C0461E6114EB451313F5106314EB4516D9
S3150800086016F51066366956F000561E611300DBB29F
S31508000870012B09D10B69002B18D014EB451313F57E
S3150800088010630E695E6111E0CB78012B0ED04B69BF
S31508000890002B0BD014F500635B6B01260F7817F05D
S315080008A00F07BE40334314F500667363CB78012BFC
S315080008B01DD114F500639B68DB050CD414EB4513B6
S315080008C013F510631B6853F0005314EB451616F521
S315080008D0106633600BE014EB451313F510631B68C1
S315080008E053F0805314EB451616F51066336014EB77
S315080008F0451313F510631B6853F0044314EB4514B2
S3150800090014F510642360CB78012B40F0A280D2B294
S3150800091000924B699BB20A78C96800F0A5F998E07D
S3150800092014EB451010F5306014EB451313F53063DE
S315080009301B69DB0CDB04036114EB451010F5306012
S3150800094014EB451313F530631B696FF3DC4303613E
S31508000950486900281AD114EB451010F5306014EBDD
S31508000960451313F530631B698E687603760B33439C
S31508000970036114EB451010F5306014EB451313F5BD
S3150800098030631B6953F40023036129E04B698868C7
S31508000990C3185B1E8868B3FBF0F014EB451313F518
S315080009A0306314EB451616F5306636690700BFB294
S315080009B0DFF874C61CEAC74C5CEA06061E6114EB2F
S315080009C0451313F5306314EB451616F5306636698C
S315080009D08F6880B200FB07F04003400B3043186174
S315080009E0D2B2012A08D1C868002805D014EB4510F0
S315080009F010F53060CA684261C87801281DD114F51F
S31508000A0000608068C0050CD414EB451010F5306002
S31508000A10006850F0005014EB451111F5306108607C
S31508000A200BE014EB451010F53060006850F080506C
S31508000A3014EB451111F53061086014EB451010F5FB
S31508000A403060006850F0044014EB451414F5306427
S31508000A5020600020F2BD0000BFFFBDFFC0ACD8007B
S31508000A6000350C00C0E1E40040420F000024F40009
S31508000A70804F12008073060120D61300A0491A0180
S31508000A8060E31600002D310140771B0040A44C019D
S31508000A90C091210000366E012075380020ABA601F2
S31508000AA0E09C410070B40B001C785978012940F08D
S31508000AB089805969002924D110EB441111F5106178
S31508000AC010EB441515F510652D696FF3DC450D61BE
S31508000AD010EB441111F5106110EB441515F510656E
S31508000AE02D6955F400250D6110EB441111F51061BF
S31508000AF010EB441515F510652D69ED0CED040D6127
S31508000B0037E010EB441111F5106110EB441515F59B
S31508000B1010652D69ED0CED040D6110EB441111F50E
S31508000B20106110EB441515F510652D696FF3DC455A
S31508000B300D6199685D69A94201D29968596110EBFE
S31508000B40441111F5106110EB441515F510652D6962
S31508000B5055F400250D6110EB441111F5106110EBE9
S31508000B60441515F510652D695E697603760B3543D0
S31508000B700D61D2B2012A09D11969002915D010EBE5
S31508000B80441111F510611A694A610EE05969002984
S31508000B900BD010F50061496B01221B7813F00F0387
S31508000BA09A40114310F50062516310EB441111F598
S31508000BB01061096851F0044110EB441010F51060FB
S31508000BC001604EE010EB441111F5306110EB44154D
S31508000BD015F530652D69ED0CED040D6110EB44112A
S31508000BE011F5306110EB441515F530652D696FF375
S31508000BF0DC450D615969002901D09968596110EBE6
S31508000C00441111F5306110EB441515F530652D6961
S31508000C1055F400250D6110EB441111F5306110EB08
S31508000C20441515F530652D699E687603760B3543B0
S31508000C300D61D2B2012A08D1D968002905D010EB76
S31508000C40441111F53061DA684A6110EB441111F567
S31508000C503061096851F0044110EB441010F530601A
S31508000C600160002070BC7047F0B4049CE4B2002C0C
S31508000C7012D19BB2DB1C9B0800250BE00E681700FF
S31508000C80FFB24FF4805404FB070717F580573E6000
S31508000C90091D6D1C9D42F1D30020F0BC704710B4AD
S31508000CA092B2D21C9208002305E010F580542468FD
S31508000CB00C60091D5B1C9342F7D3080010BC7047F3
S31508000CC0020008784978012921D112EB401111F563
S31508000CD01061096800290DD400280BD012EB4011C9
S31508000CE011F51061096831F0804112EB401313F5D4
S31508000CF01063196012EB401111F51061096851F47F
S31508000D00001112EB401212F51062116020E012EB8E
S31508000D10401111F53061096800290DD400280BD05F
S31508000D2012EB401111F53061096831F0804112EB80
S31508000D30401313F53063196012EB401111F5306159
S31508000D40096851F4001112EB401212F53062116075
S31508000D500020704710B40A784B78012B1ED110EB8F
S31508000D60421313F510631B6833F4001310EB421497
S31508000D7014F510642360CB78032B02D0C9780229B6
S31508000D802AD110EB421111F51061096851F0805112
S31508000D9010EB421010F5106001601DE010EB4213D5
S31508000DA013F530631B6833F4001310EB421414F583
S31508000DB030642360CB78032B02D0C97802290BD183
S31508000DC010EB421111F53061096851F0805110EBB2
S31508000DD0421010F530600160002010BC704710B555
S31508000DE00400200000210CE04FF67F3210EB41137F
S31508000DF013F510639A6010EB411313F530639A608C
S31508000E00491C0F29F0D3002110F500621161002159
S31508000E1010F500625161002110F50060C1612000E3
S31508000E20FFF7BAFB0100C9B2002901D0C0B20AE037
S31508000E3010212000FFF79FFB0100C9B2002901D04D
S31508000E40C0B200E0C0B210BD10F50062126832F4FC
S31508000E50FE6210F500631A6010F500621268C9B2E6
S31508000E60090111F4FE61114310F5006001600020CC
S31508000E70704780B510F50061496831F0020110F538
S31508000E8000604160032000F0D3F8002002BD80B561
S31508000E9010F50061496851F0020110F500604160E3
S31508000EA0032000F0C5F8002002BD010048698969E1
S31508000EB008407047010011F50060806911F500616E
S31508000EC0C9690840000C7047010011F50060806987
S31508000ED011F50061C969084080B270470200C9B2BD
S31508000EE012EB411010F53060806812F50062516906
S31508000EF00840704710B410F50062126910F50063D7
S31508000F005B6B11F00F04E340DB0113F080031A4317
S31508000F10C9B210EB411010F510608068104010BC83
S31508000F207047406910F00100704710F510610968B4
S31508000F30C90AC90210F51062116010F500618968C6
S31508000F4011F00601042907D110F51061096851F05E
S31508000F50030110F51062116010F50061496851F43B
S31508000F60807110F5006041600020704710B40300DE
S31508000F70006CDFF8B840A04206D313F5306000686D
S31508000F80002801D500202AE0002013F530642061EE
S31508000F9013F53060006950F4002013F530642061C1
S31508000FA013F53060006950F0180013F530642061BD
S31508000FB013F53060006950F0C04013F530642061C5
S31508000FC0C9B201290AD113F53060426113F53060C0
S31508000FD0006850F0802013F530631860002010BCBC
S31508000FE070470021491C0D4A91420FD20369002B14
S31508000FF0F8D50021036953F001030361491C9142A6
S3150800100006D20369DB07F9D4002070470320FCE702
S315080010100320FAE70001800000383C80410D0300F8
S31508001020007833EC0078F3EF0000F81F0B30544FCC
S3150800103038B5040000F03EF8050014F1010F02D09F
S3150800104004480078241800F035F8401BA042FAD36B
S3150800105031BD00BFBD00002080B500F00DF8104876
S315080010601049086000201049086005200F490860EB
S3150800107000200F49086001BD00200C490860704730
S315080010800A480068C00303D509480168491C01607D
S31508001090704780B5FFF7F4FF0548006802BD0000F9
S315080010A0BF4B030014E000E018E000E010E000E0A9
S315080010B00410002080B5FFF7ECFF02BD704730B47E
S315080010C0002513E050F8042BD30744BFA9F1010308
S315080010D09A18091F042942F8045BFAD213468C07AA
S315080010E044BF15809B1CC90748BF1D7050F8041BD8
S315080010F00029E7D130BC704710B58AB00400002C2F
S3150800110001D10120B0E094F8BD03002805D10020E4
S3150800111084F8BC03200000F051FE032084F8BD03C8
S315080011202068FFF7F8F8211D83B06846342200F0DE
S3150800113047FE0EBC2068FFF747F8002804D00220B7
S3150800114084F8BD0301208FE000212068FFF7E9F845
S31508001150002130E01C200A00D2B242432244012377
S3150800116082F83D300A00D2B24243224482F83C104B
S315080011700A00D2B2424322440B00DBB2A2F8423044
S315080011800A00D2B242432244002382F83F300A00C2
S31508001190D2B242432244002353640A00D2B24243E5
S315080011A02244002393640A00D2B200FB02F02044D2
S315080011B000220265491C0800C0B262689042C9D381
S315080011C000212BE01C200A00D2B24243224400230D
S315080011D082F8FD310A00D2B24243224482F8FC1159
S315080011E00A00D2B242432244002382F8FF310A00A1
S315080011F0D2B2424322440023C2F804320A00D2B2D1
S31508001200424322440023C2F808320A00D2B200FB45
S3150800121002F020440022C0F81022491C0800C0B27F
S3150800122062689042CED3211D83B06846342200F00E
S31508001230C7FD0EBC2068FFF790F8002804D00220EE
S3150800124084F8BD0301200FE0002084F8380001204F
S3150800125084F8BD03606A012802D1200000F029FE47
S315080012602068FFF714FE00200AB010BD10B5040070
S31508001270002C01D101200CE0032084F8BD032000D6
S3150800128000F01EF8200000F028FE002084F8BD03B8
S31508001290002010BD10B5040094F8BC03012801D144
S315080012A002200CE0012084F8BC032068FFF7E1FD6A
S315080012B02068FFF72AF8002084F8BC03002010BD38
S315080012C010B5040094F8BC03012801D1022016E0E9
S315080012D0012084F8BC032068FFF71DF82068FFF793
S315080012E07EFD002804D0002084F8BC03012006E017
S315080012F02068FFF7CCFD002084F8BC03002010BD51
S315080013002DE9F84306003768B84600243068FFF729
S3150800131008FE002840F06C823068FFF7C6FD0028FA
S3150800132000F066823068FFF7C0FD800705D5306893
S31508001330406910F00200316848613068FFF7B5FD72
S31508001340000350D500243068FFF7B4FD050048E0D7
S31508001350E80744D52100C9B23068FFF7BFFD8146CA
S315080013605FEAC97009D518EB441010F53060012101
S3150800137081602100300000F046FC5FEA097009D55B
S315080013802100300000F0DEFC18EB441010F5306048
S31508001390082181605FEAC96005D518EB441010F58D
S315080013A03060102181605FEA89600ED530690128B6
S315080013B005D116F5717201213068FFF7D7FD18EBD4
S315080013C0441010F53060202181605FEA894006D517
S315080013D018EB441010F530604FF400518160641C1E
S315080013E06D08002DB4D13068FFF75FFD40037AD54C
S315080013F03068FFF769FD0500002472E0E8076ED53E
S315080014002100C9B23068FFF775FD81465FEAC970E9
S315080014103AD5012114F00F0011FA00F018F5006111
S31508001420496B31EA000018F50061486318EB44106F
S3150800143010F5106001218160306901280DD11C204A
S3150800144000FB04F13144896C00FB04F23244526C0F
S31508001450114400FB04F0304481642100C9B2300015
S3150800146000F053FD306901280ED1002C0CD11C2048
S3150800147000FB04F03044006D002805D116F57172A2
S3150800148001213068FFF772FD5FEA097005D518EB90
S31508001490441010F51060082181605FEAC96005D51F
S315080014A018EB441010F51060102181605FEA49605E
S315080014B005D518EB441010F51060402181605FEAED
S315080014C0897005D518EB441010F51060022181606B
S315080014D05FEA096003D52100300000F020FB641C98
S315080014E06D08002D8AD13068FFF7DFFC00281CD56F
S315080014F018F5006040684008400018F5006148602B
S3150800150096F8F403012807D1002086F8F403002191
S31508001510300000F0E1FC02E0300000F041FD3068E8
S31508001520406910F00040316848613068FFF7BDFC3B
S3150800153000050DD518F500608068C00702D5300093
S3150800154000F013FD3068406910F4006031684861A6
S315080015503068FFF7AAFC00011AD53068406910F018
S3150800156000603168486196F8F40300280DD101201F
S3150800157086F8F4033068406DC0F38300C6F8F803B4
S315080015800121300000F0A8FC02E0300000F0EDFC7C
S315080015903068FFF78AFCC0047BD518F50060406800
S315080015A04008400018F50061486010213068FEF7D1
S315080015B0E2FF002024E04FF67F3118EB401212F5C7
S315080015C01062916018EB401212F51062126832F43C
S315080015D0001218EB401313F510631A6018EB40124B
S315080015E012F53062916018EB401111F53061096807
S315080015F031F4001118EB401212F530621160401CEC
S3150800160071688842D7D318F50060C06950F0011098
S3150800161018F50061C861306B002812D018F5006013
S31508001620D0F8840050F00B0018F50061C1F884006A
S3150800163018F50060406C50F00B0018F5006148641E
S3150800164011E018F50060406940F4005050F02B0096
S3150800165018F50061486118F50060006950F00B0044
S3150800166018F50061086118F50060006830F4FE603E
S3150800167018F50068C8F8000016F571723169C9B224
S315080016803068FFF773FC3068406910F480503168A1
S3150800169048613068FFF709FC800417D53068FFF702
S315080016A044FC3068FEF791FFF06000F09FFD0100F2
S315080016B0F268D2B23068FEF7BFFD300000F039FCA0
S315080016C03068406910F40050316848613068FFF7A7
S315080016D0ECFBC0063FD53068806930F010003168F1
S315080016E08861D7F8208018F00F011C20414306EBCB
S315080016F0010010F5FE75C8F34340022816D147F6D7
S31508001700F07018EA000F20D0C8F30A1292B2E968FE
S315080017103800FFF7C4FAE868C8F30A110844E86015
S31508001720A969C8F30A104118A9610EE0C8F3434035
S3150800173006280AD1082216F571713800FFF7AFFAA4
S31508001740A969C8F30A104118A9613068806950F080
S315080017501000316888613068FFF7A7FB000708D5D5
S31508001760300000F0E0FB3068406910F0080031688E
S3150800177048613068FFF799FBC0020AD52100C9B253
S31508001780300000F01DFC3068406910F480103168A4
S3150800179048613068FFF789FB80020AD52100C9B283
S315080017A0300000F006FC3068406910F4001031681B
S315080017B048613068FFF779FB400008D5300000F033
S315080017C006FC3068406910F080403168486130682E
S315080017D0FFF76BFB40070BD530684468600702D5F6
S315080017E0300000F0FEFB306840680443306844600F
S315080017F0BDE8F18310B5040094F8BC03012801D1B3
S31508001800022009E0012084F8BC032068FFF731FBB9
S31508001810002084F8BC03002010BD10B5040094F81D
S31508001820BC03012801D1022009E0012084F8BC0389
S315080018302068FFF72CFB002084F8BC03002010BDAD
S3150800184010B5040094F8BC03012801D102200CE06D
S31508001850012084F8BC0384F83810C9B22068FFF761
S31508001860F3FA002084F8BC03002010BD70B505000B
S3150800187000260800C0B200060CD50C00E4B214F02D
S315080018800F041C20444305EB040010F13C0401201E
S3150800189060700BE00C00E4B214F00F041C20444303
S315080018A005EB040010F5FE740020607011F00F01BE
S315080018B0217092B2A260E3706078002801D0207887
S315080018C0E080DBB2022B01D10020207195F8BC0321
S315080018D0012801D102200BE0012085F8BC03210074
S315080018E02868FEF784FE002085F8BC033000C0B2E5
S315080018F070BD10B504000800C0B200060BD50A007A
S31508001900D2B212F00F021C20424304EB02003C3014
S31508001910012242700BE00A00D2B212F00F021C201C
S31508001920424304EB020010F5FE700022427011F0EB
S315080019300F01017094F8BC13012901D102200AE0B5
S31508001940012184F8BC1301002068FEF7ADFE0020D3
S3150800195084F8BC03002010BD38B51C000D00EDB29C
S3150800196015F00F051C235D4300EB050313F5FE7305
S31508001970DA605C6100249C6100245C7011F00F043D
S315080019801C700469012C00D11A6111F00F0F06D1E1
S315080019900269D2B219000068FFF784F805E0026907
S315080019A0D2B219000068FEF7D7FE002032BDC9B2D0
S315080019B011F00F011C2251430844D0F81402704755
S315080019C038B51C000D00EDB215F00F051C235D435C
S315080019D000EB05033C33DA605C6100249C6101245A
S315080019E05C7011F00F041C700469012C00D11A6197
S315080019F011F00F0F06D10269D2B219000068FFF77D
S31508001A0051F805E00269D2B219000068FEF7A4FE93
S31508001A10002032BD38B504000D0060682900C9B23F
S31508001A2011F00F01884201D2012039E02800C0B226
S31508001A3000060CD52900C9B211F00F011C2041433C
S31508001A4004EB010010F13C010120487009E029006F
S31508001A50C9B21C20414304EB010010F5FE710020B9
S31508001A6048700120887015F00F00087094F8BC03C0
S31508001A70012801D1022013E0012084F8BC03206864
S31508001A80FFF71EF915F00F0F06D114F571722169CB
S31508001A90C9B22068FFF76AFA002084F8BC03002060
S31508001AA032BD10B5040060680A00D2B212F00F0207
S31508001AB0904201D2012031E00800C0B200060BD5E1
S31508001AC00A00D2B212F00F021C20424304EB0200B5
S31508001AD03C30012242700BE00A00D2B212F00F022B
S31508001AE01C20424304EB020010F5FE7000224270EF
S31508001AF00022827011F00F01017094F8BC130129BD
S31508001B0001D102200AE0012184F8BC1301002068F3
S31508001B10FFF720F9002084F8BC03002010BD2DE94A
S31508001B20FC4704000D00266837001C2000FB05F062
S31508001B30204410F13C08D8F81400D8F81810884248
S31508001B4001D201205DE0D8F81400D8F81890B0EB5F
S31508001B500909D8F80800484501D2D8F8089019F1BB
S31508001B6003095FEA990926E0D8F81400D8F818A0FE
S31508001B70B0EB0A0AD8F80800504501D2D8F808A0F0
S31508001B801AF103095FEA99092069C0B20090534621
S31508001B909BB22A00D2B2D8F80C103000FFF764F8CE
S31508001BA0D8F80C005044C8F80C00D8F818001AEBFE
S31508001BB0000AC8F818A017EB451010F510608069E0
S31508001BC080B2484509D3D8F81800D8F814108842C6
S31508001BD003D2D8F814000028C6D1D8F81800D8F8C7
S31508001BE0141088420CD3012015F00F0510FA05F5DC
S31508001BF017F50060406B30EA050517F500677D6349
S31508001C000020BDE8F687F8B505000C002868060030
S31508001C10006C16EB441111F5306189682A69012AAE
S31508001C206ED10A071BD5634A904208D3080406D525
S31508001C3016EB441010F530604FF40041816028001F
S31508001C4000F04CF915F5717201212868FFF78EF935
S31508001C5016EB441616F530660820B06070E08A0662
S31508001C6006D516EB441616F530662020B06067E0F8
S31508001C7011F0280F64D14F4A904209D3080407D5BA
S31508001C8016EB441616F530664FF40040B06057E080
S31508001C901C2707FB04F02844D0F8040216EB441668
S31508001CA016F5306631694903490B401A07FB04F1FA
S31508001CB02944C1F8140207FB04F02844D0F80802A6
S31508001CC007FB04F12944D1F80412084407FB04F180
S31508001CD02944C1F808022100C9B2280000F006F913
S31508001CE0002C2DD17C4305EB0400D0F81002002807
S31508001CF026D115F5717201212868FFF737F91FE01B
S31508001D002D4A904217D1080407D516EB441616F546
S31508001D1030664FF40040B06012E0880605D516EB31
S31508001D20441616F530662020B0602100C9B2280096
S31508001D3000F0DCF804E02100C9B2280000F0D6F86B
S31508001D400020F2BD38B5040022681000156C10EBAF
S31508001D50411212F5306292682369012B0CD1154B9A
S31508001D609D4215D3120413D510EB411010F53060BF
S31508001D704FF4004181600BE00F4B9D4208D11204DD
S31508001D8006D510EB411010F530604FF40041816024
S31508001D90200000F0A3F80748854208D320690128E7
S31508001DA005D114F5717201212068FFF7DFF80020CC
S31508001DB032BD00000B30544F0A31544F70470000B3
S31508001DC0103A07D330B4B1E83810103AA0E8381002
S31508001DD0F9D230BC530724BFB1E80810A0E80810B0
S31508001DE044BF51F8043B40F8043BD20724BF31F8FE
S31508001DF0022B20F8022B44BF0B7803707047121F82
S31508001E0017D35B0009D151F8043B20F8023B1B0CA1
S31508001E10121F20F8023BF6D20BE051F8043B00F8FB
S31508001E20013B1B0A20F8023B1B0C121F00F8013B62
S31508001E30F3D238BF121D521E24BF11F8013B00F819
S31508001E40013BF8D87047000070B403685B6A0C0061
S31508001E50E4B2002C05D192B253EA024300688362C9
S31508001E601FE00468A46A13EB1443002409E005681C
S31508001E702600F6B205EB8605D5F8045113EB154393
S31508001E80641C2500EDB20E00F6B2761EB542EED3FE
S31508001E900068C9B200EB810092B253EA0243C0F867
S31508001EA00031002070BC704789B20068416200208A
S31508001EB0704701680122C0F8FC23002280F8F42349
S31508001EC0886950F000608861486D40F0805050F095
S31508001ED003004865002070477047704780B510F5C5
S31508001EE07171D0F8000400F0DDF901BD80B50B0072
S31508001EF0DBB21C22534300EB0302D2F80822C9B214
S31508001F00D0F8000400F000FA01BD80B50B00DBB282
S31508001F101C22534300EB0302926CC9B2D0F80004AA
S31508001F2000F045FA01BD80B5D0F8000400F003FBC7
S31508001F3001BD38B504000125E068002801D1002557
S31508001F4008E0E068022801D1012503E0912146480E
S31508001F5000F013FB2900C9B2D4F8000400F0D9FA3E
S31508001F60D4F8000400F0A5FA31BD10B50400D4F881
S31508001F70000400F0D1FA206810F56060006850F09F
S31508001F800100216811F560610860206A002804D004
S31508001F903648016851F00601016000F017FB10BDD4
S31508001FA010B5040000F013FBD4F8000400F0BDFAE5
S31508001FB010BD80B5C9B2D0F8000400F0CEFA01BD54
S31508001FC080B5C9B2D0F8000400F0C5FA01BD10B555
S31508001FD00400012000F0F9FAD4F8000400F0BFFA72
S31508001FE010BD10B50400002000F0EFFAD4F8000484
S31508001FF000F0B7FA10BD10B50178002931D11C4C94
S31508002000C4F80004C0F898425FF0A040206006209B
S3150800201060600220E060002020610220A0610120AB
S31508002020E06100202062002060620020E06200205B
S3150800203020632000FFF760F8002804D040F225113D
S31508002040094800F09AFA80212000FFF72DFF402268
S3150800205000212000FFF7F8FE802201212000FFF76B
S31508002060F3FE002010BD0000645A000810ED00E0E1
S31508002070C000002080B500210021D0F89802FFF7A3
S31508002080F5F8C0B200F09DF8C0B202BD80B50021D7
S315080020900021D0F89802FFF7FDF8C0B200F091F8D9
S315080020A0C0B202BD80B500210021D0F89802FFF722
S315080020B007F9C0B200F085F8C0B202BD10B51C0021
S315080020C0002300231300DBB2220092B2C9B2D0F873
S315080020D09802FFF7CBFBC0B200F073F8C0B210BD90
S315080020E080B500220022C9B2D0F89802FFF701FC99
S315080020F0C0B200F066F8C0B202BD80B50022002268
S31508002100C9B2D0F89802FFF785FCC0B200F059F8BA
S31508002110C0B202BD80B500220022C9B2D0F898022A
S31508002120FFF7BFFCC0B200F04CF8C0B202BDD0F851
S3150800213098220800C0B2000609D5C9B211F07F017D
S315080021401C20414302EB010090F83E0008E0C9B2AA
S3150800215011F07F011C20414302EB010090F8FE01BB
S31508002160704780B500220022C9B2D0F89802FFF75E
S3150800217067FBC0B200F025F8C0B202BD10B5002456
S3150800218000249BB2C9B2D0F89802FFF719FCC0B276
S3150800219000F017F8C0B210BD10B5002400249BB299
S315080021A0C9B2D0F89802FFF7D7FBC0B200F009F819
S315080021B0C0B210BD80B5C9B2D0F89802FFF7F7FBD8
S315080021C002BD0021C0B2002805D0022807D004D3DA
S315080021D0032806D007E0002006E0022004E00120DC
S315080021E002E0022000E00220C0B270470148006801
S315080021F0704700000400002080B5002801D10220A5
S3150800220011E0D0F88C32002B02D00023C0F88C32B3
S31508002210002901D0C0F88812012180F874120270D2
S31508002220FFF7E9FE002002BD10B50400012084F87E
S3150800223074026168C9B22000D4F88C2252689047AB
S315080022402000FFF72FFF2000FFF714FF002010BD26
S315080022500022002903D0C0F88C12002000E00220DA
S31508002260C0B2704780B5FFF711FF002002BD0020FD
S31508002270704710B50224D0F88C22002A07D0C9B2BC
S31508002280D0F88C2212689047002800D1002420003C
S31508002290C0B210BD80B5C9B2D0F88C22526890473A
S315080022A0002002BD10B5040014F5207000F0C4FC2F
S315080022B00120C4F86C02B4F88602C4F8700294F8D7
S315080022C0800210F01F00002803D002280DD006D384
S315080022D011E014F52071200000F07AF912E014F5E7
S315080022E02071200000F0B1F90CE014F520712000EF
S315080022F000F0E1F906E094F8801211F08001200060
S31508002300FFF7FBFE002010BD10B5040010000A0000
S31508002310D2B2002A39D114F5A072D4F86C12032966
S3150800232027D11169D368994211D2D36811695B1A0A
S31508002330D360D1681369994201D2D26800E0126964
S3150800234092B20100200000F0E2FC002010BDD4F893
S315080023508C020069002808D094F87402032804D176
S315080023602000D4F88C1209698847200000F0D8FCB0
S31508002370EBE7D4F86C020528E7D10020C4F86C0214
S3150800238000212000FFF7B9FEDFE7D4F88C02806948
S3150800239000280AD094F87402032806D1C9B220008E
S315080023A0D4F88C2292699047CFE70220CEE710B581
S315080023B0040010000A00D2B2002A68D114F11402EF
S315080023C0D4F86C1202294AD11169D368994210D2FD
S315080023D0D36811695B1AD360D26892B201002000F3
S315080023E000F08CFC0023002200212000FFF7D4FE19
S315080023F041E090681169B0FBF1F301FB1300002876
S3150800240017D190681169884213D39068D4F870126E
S3150800241088420ED200220021200000F06FFC002026
S31508002420C4F870020023002200212000FFF7B4FE42
S3150800243021E0D4F88C02C068002808D094F8740209
S31508002440032804D12000D4F88C12C9688847802153
S315080024502000FFF752FE200000F06DFC0BE0D4F8D8
S315080024606C02042803D0D4F86C02002803D180211A
S315080024702000FFF742FE94F87802012805D12000D3
S31508002480FFF7F5FE002084F87802002010BDD4F886
S315080024908C02406900280AD094F87402032806D1F1
S315080024A0C9B22000D4F88C2252699047EDE7022081
S315080024B0ECE710B504004023002200212000FFF7B6
S315080024C0FDFD0120C4F844014020C4F85001402312
S315080024D0002280212000FFF7F1FD0120A0614020A5
S315080024E06062012084F874020020C4F86C0200209F
S315080024F060600020C4F87C02D4F89002002806D058
S315080025006168C9B22000D4F88C225268904700202E
S3150800251010BD01740020704790F8741280F8751287
S31508002520042180F874120020704790F8751280F81C
S3150800253074120020704780B590F87412032908D1E8
S31508002540D0F88C12C969002903D0D0F88C12C96951
S315080025508847002002BD00207047002070470020F1
S31508002560704780B5012180F874124168C9B2D0F865
S315080025708C2252689047002002BD80B500F0EAFB25
S31508002580FCE7000000690840884201D1012000E00C
S315080025900020C0B2704780B54FF400510548FFF7D8
S315080025A0F1FF002801D0002002E000F0FEFB012028
S315080025B002BD00000008024080B5642000F0D3FB8D
S315080025C001BD80B500F0D2FB01BD7047704770476A
S315080025D010B500240A7812F06002002A08D0202AD2
S315080025E001D0402A2CD1D0F88C229268904729E055
S315080025F04A78002A18D0012A1CD0032A17D0052A9F
S3150800260009D0062A04D0082A0BD0092A06D014E0D5
S3150800261000F077F913E000F01CFA10E000F048FA31
S315080026200DE000F0AFFA0AE000F0CBFA07E000F0A0
S31508002630E7FA04E000F0EEFA01E000F011FB01E031
S3150800264000F00EFB2000C0B210BD38B504000D0026
S315080026500020287810F06000002803D0202801D038
S31508002660402822D194F87402401E022818D82879E6
S31508002670022810D229002000D4F88C2292689047AC
S315080026800100E88800280AD1C9B2002907D120002C
S3150800269000F046FB03E02900200000F0E1FA03E021
S315080026A02900200000F0DCFA03E02900200000F0F1
S315080026B0D7FA002032BD70B50500002488880A784C
S315080026C012F06002002A0AD0202A02D0402A40F0DE
S315080026D012812800D5F88C22926890470EE10A7874
S315080026E012F06002202A06D12800D5F88C229268BA
S315080026F09047C0B204E14A78002A6CD0012A3AD041
S31508002700032A40F0F48095F87422022A02D0032A9C
S3150800271016D02CE00200D2B2002A0DD00200D2B2A6
S31508002720802A09D00100C9B22800FFF7E6FC8021FB
S315080027302800FFF7E2FC02E0280000F091FA19E011
S315080027404A88002A0FD10200D2B2002A0BD0020012
S31508002750D2B2802A07D0C988002904D10100C9B29B
S315080027602800FFF7CAFC280000F0DAFA02E0280081
S3150800277000F076FABEE095F87422022A02D0032AFF
S3150800278016D024E00200D2B2002A0DD00200D2B23E
S31508002790802A09D00100C9B22800FFF7AEFC8021C3
S315080027A02800FFF7AAFC02E0280000F059FA11E019
S315080027B0498800290AD110F07F0F04D00100C9B258
S315080027C02800FFF7A7FC280000F0AAFA02E0280074
S315080027D000F046FA8EE095F87422022A02D0032AFF
S315080027E028D080E00200D2B2002A07D00200D2B276
S315080027F0802A03D0280000F033FA77E00100C9B236
S31508002800090608D5C0B210F07F00142148432844B1
S3150800281010F1140107E0C0B210F07F0014214843FC
S31508002820284410F5A071002008600222280000F054
S3150800283053FA5BE00200D2B212060ED50300DBB2F1
S3150800284013F00F031422534305EB03029269002A7F
S3150800285013D1280000F004FA48E00300DBB213F0B5
S315080028600F031422534305EB0302D2F84421002A2E
S3150800287003D1280000F0F4F938E00100C9B20906CE
S315080028800AD50200D2B212F07F0214214A4305EBA0
S31508002890020111F1140609E00200D2B212F07F0219
S315080028A014214A4305EB020111F5A0760100C9B2CD
S315080028B0002903D00100C9B2802902D10020306066
S315080028C00BE00100C9B22800FFF731FC002802D04E
S315080028D00120306001E0002030600222310028002B
S315080028E000F0FAF902E0280000F0BAF902E0280040
S315080028F000F0B6F902E0280000F0B2F92000C0B2F4
S3150800290070BD38B504000D00688880B2000AC0B2F0
S31508002910012808D002281BD003282CD0062865D009
S31508002920072871D080E06946207CD4F8882212688E
S315080029309047BDF80010002900F08480E988002936
S3150800294000F08080BDF80010EA88914271D273E0E9
S31508002950207C002807D16846D4F88C12896A8847F3
S315080029600221417006E06846D4F88C12C96A884785
S3150800297002214170DDE7A878002808D0022814D083
S315080029800CD304281FD017D3052823D029E069467D
S31508002990207CD4F8882252689047CAE76946207C8A
S315080029A0D4F8882292689047F7E76946207CD4F8DD
S315080029B08822D2689047F0E76946207CD4F88822B6
S315080029C012699047E9E76946207CD4F8882252695B
S315080029D09047E2E76946207CD4F8882292699047B6
S315080029E0DBE72900200000F03BF931E0207C0028D5
S315080029F005D16846D4F88C12496B884799E72900AF
S31508002A00200000F02DF923E0207C002807D1684635
S31508002A10D4F88C12096B88470721417089E7290089
S31508002A20200000F01DF913E02900200000F018F935
S31508002A300EE0E988ADF80010BDF80020010020007E
S31508002A4000F04AF9E888002802D1200000F068F969
S31508002A5031BD38B505008888002825D1C8880028E2
S31508002A6022D1488880281FD28C7814F07F0495F8E4
S31508002A707402032803D1280000F0F2F817E085F85D
S31508002A8076422100C9B22800FFF76BFB280000F048
S31508002A9047F9E4B2002C03D0022085F8740206E058
S31508002AA0012085F8740202E0280000F0D9F831BD4B
S31508002AB070B504000D00324E6888307030780228F0
S31508002AC004D32900200000F0CBF857E094F87402EC
S31508002AD0022802D003281BD048E03078002813D0FB
S31508002AE030786060032084F8740231782000FFF79C
S31508002AF0C0FB022804D12900200000F0B1F83DE00F
S31508002B00200000F00DF902E0200000F009F935E098
S31508002B10307800280CD1022084F87402307860607E
S31508002B2031782000FFF7B6FB200000F0F9F81CE02A
S31508002B3030786168884215D06168C9B22000FFF70D
S31508002B40A9FB3078606031782000FFF792FB0228F5
S31508002B5004D12900200000F083F80FE0200000F0DF
S31508002B60DFF802E0200000F0DBF807E0290020008B
S31508002B7000F076F831782000FFF78CFB70BD000076
S31508002B801810002080B5CA88012A02D000F068F81B
S31508002B9016E090F87422521E012A02D9921E08D015
S31508002BA00CE000218160012210F1080100F094F880
S31508002BB006E00122011D00F08FF801E000F050F850
S31508002BC001BD80B590F87422521E022A15D8CA880B
S31508002BD0022A02D000F044F811E00121C160D0F8C1
S31508002BE07C12002903D0C16851F00201C16002229B
S31508002BF010F10C0100F070F801E000F031F801BDA9
S31508002C0080B54988012904D10121C0F87C1200F059
S31508002C1087F801BD80B590F87422521E022A08D89A
S31508002C204988012904D10021C0F87C1200F078F8FF
S31508002C3001E000F015F801BD0A7802704A78427082
S31508002C408A78CB781B029A1842800A794B791B023C
S31508002C509A1882808A79C97909028918C1807047C9
S31508002C6010B5040080212000FFF747FA0021200054
S31508002C70FFF743FA10BDF8B504000D00170000264B
S31508002C80002C1ED0200000F01DF84000801C388063
S31508002C9038783100C9B26854761C03203100C9B2AD
S31508002CA06854761C0AE020783100C9B26854641C5E
S31508002CB0761C00203100C9B26854761C207800289A
S31508002CC0F1D1F1BD0200002001E0401C521C117830
S31508002CD00029FAD1C0B2704780B513000222C0F8A5
S31508002CE06C221A0092B2C2611A0092B202629BB2B8
S31508002CF00A000021FFF742FA002002BD80B5130042
S31508002D009BB20A000021FFF739FA002002BD80B500
S31508002D1013009BB20A000021FFF73EFA002002BD0D
S31508002D2080B50421C0F86C12002300220021FFF7A9
S31508002D3025FA002002BD80B50521C0F86C120023D3
S31508002D4000220021FFF728FA002002BD80B5FFF710
S31508002D5033FC01BD80B5FFF734FC01BD81617047C6
S31508002D6009048161704714490880704710B5FEF759
S31508002D7090F9124C2168884216D311490878002820
S31508002D8006D10120087080210E48FFF7E7FF05E00D
S31508002D900020087080210B48FFF7E2FFFEF779F95B
S31508002DA0054909884018206010BD80B5802105486E
S31508002DB0FFF7D6FF01BD000010100020FC0F002011
S31508002DC0131000200004024038B50400002C01D17D
S31508002DD00120AEE094F82000002802D1200000F07F
S31508002DE0B0FA2068006830F0020021680860FEF733
S31508002DF061F905002068406880070DD5FEF75AF985
S31508002E00401B0B28F6D3606A50F400306062052038
S31508002E1084F8200001208CE02068006850F001004A
S31508002E2021680860FEF746F9050020684068C00773
S31508002E300DD4FEF73FF9401B0B28F6D3606A50F411
S31508002E4000306062052084F82000012071E0207EB1
S31508002E50012806D12068006850F0800021680860C3
S31508002E6005E02068006830F0800021680860607E10
S31508002E70012806D12068006850F0400021680860E3
S31508002E8005E02068006830F0400021680860A07EF0
S31508002E90012806D12068006850F0200021680860E3
S31508002EA005E02068006830F0200021680860E07EB0
S31508002EB0012806D12068006830F0100021680860F3
S31508002EC005E02068006850F0100021680860207F3F
S31508002ED0012806D12068006850F0080021680860BB
S31508002EE005E02068006830F0080021680860607F07
S31508002EF0012806D12068006850F00400216808609F
S31508002F0005E02068006830F0040021680860A168C0
S31508002F10E068014320690143606901436068401E17
S31508002F2001432068C16100206062012084F8200006
S31508002F30002032BD30B4026890F820201300DBB2BE
S31508002F40012B03D0D2B2022A40F07F80594AD2F828
S31508002F50000250F00100C2F80002D2F8000230F474
S31508002F607C50C2F80002D2F800024B6A50EA0320ED
S31508002F70C2F8000201200B7D13F01F0310FA03F3B9
S31508002F80D2F81C029843C2F81C02C869002816D158
S31508002F90D2F80C029843C2F80C02486902EBC0004A
S31508002FA0CC684D68C5EA0444C0F84042486902EB5B
S31508002FB0C0008C680D68C5EA0444C0F84442C86974
S31508002FC0012816D1D2F80C021843C2F80C02486937
S31508002FD002EBC0000C684D68C5EA0444C0F84042DC
S31508002FE0486902EBC0008C68CD68C5EA0444C0F89D
S31508002FF044428869002805D1D2F804029843C2F8E9
S31508003000040204E0D2F804021843C2F8040208696C
S31508003010002805D1D2F814029843C2F8140204E035
S31508003020D2F814021843C2F81402086A012804D117
S31508003030D2F81C020343C2F81C32D2F80002400838
S315080030404000C2F80002002004E0416A51F48021E1
S315080030504162012030BC704738B5040094F820005E
S31508003060012821D1022084F8200020680068400841
S31508003070400021680860FEF71DF8050020684068D2
S31508003080C0070DD5FEF716F8401B0B28F6D3606A65
S3150800309050F400306062052084F82000012008E022
S315080030A000206062002004E0606A50F4002060623C
S315080030B0012032BD0064004070B490F820500468C6
S315080030C0A6688C68002CFFD02C00E4B2012C02D034
S315080030D0EDB2022D6ED116F0E05F65D0C6F301643D
S315080030E0032C05D3416A51F400014162012066E0D0
S315080030F00125A5401D608B68002B09D10B68CD689A
S3150800310055EA4355036826013344C3F880510AE05B
S315080031104B688D6855EAC305CB681D4303682601CD
S315080031203344C3F880510B69056826013544C5F850
S315080031308431097D01290BD1016823011944D1F88D
S31508003140841151F48071036825012B44C3F8841156
S31508003150D17993791B0453EA0163517953EA012320
S3150800316011790B43016825012944C1F88C31D178BE
S3150800317093781B0453EA0163517853EA01231178C3
S315080031800B43016822011144C1F888310168220104
S315080031901144D1F8801151F0010100682201104450
S315080031A0C0F8801100200AE0416A51F4001141621A
S315080031B0012004E0416A51F480214162012070BC7B
S315080031C0704710B40200002092F820301C00E4B2C8
S315080031D0012C02D0DBB2022B07D11268926812EAE0
S315080031E08162B2EB816F00D0012010BC704730B409
S315080031F090F820402500EDB2012D03D0E4B2022C50
S3150800320040F0988000290AD10468E46814F0030F96
S3150800321010D1416A51F40011416201208FE004681F
S31508003220246914F0030F05D1416A51F40011416273
S31508003230012084E004680D012C44D4F8B04114F050
S31508003240040494609468002C07D104680D012C448A
S31508003250D4F8B041640D146006E004680D012C44EE
S31508003260D4F8B041E408546004680D012C44D4F83D
S31508003270B041C4F34004D46004680D012C44D4F86A
S31508003280B44114F00F04146104680D012C44D4F8F9
S31508003290B441C4F30724946104680D012C44D4F89E
S315080032A0B441240C546102680C012244D2F8B821B6
S315080032B01A7002680C012244D2F8B821120A5A7010
S315080032C002680C012244D2F8B821120C9A700268DE
S315080032D00C012244D2F8B821120EDA7002680C01E9
S315080032E02244D2F8BC211A7102680C012244D2F891
S315080032F0BC21120A5A7102680C012244D2F8BC2178
S31508003300120C9A7102680C012244D2F8BC21120EE2
S31508003310DA71002906D10168C96851F020010068F0
S31508003320C16005E00168096951F020010068016182
S31508003330002004E0416A51F480214162012030BC3A
S3150800334070477047DFF8D804016851F00101016041
S315080033507047DFF8CC040068400810F00100704799
S31508003360DFF8BC140A6832F0F80252EAC0020A60B2
S315080033707047DFF8B0040068400810F00100704795
S31508003380DFF8A804006810F00C007047DFF89C040A
S31508003390006810F0F0007047DFF89004006810F439
S315080033A0E0507047DFF88404006810F46040704706
S315080033B00100DFF87C040068084050EA01407047C5
S315080033C00100DFF86C040068084050EA01407047C5
S315080033D0DFF84C040068400E10F001007047DFF873
S315080033E05404006810F480007047DFF84804006849
S315080033F0C0F388107047DFF83C04006810F44030CA
S315080034007047DFF83004006810F03F007047DFF8B7
S3150800341010040068C00E10F001007047DFF80004C1
S315080034200068400F10F00100704710B55FF0FF34D8
S31508003430FFF788FFFFF78DFF0128FBD10020DFF893
S31508003440EC130860DFF8F8030440DFF8D4030460DF
S315080034501020FFF785FFFFF7BBFF0028FBD1FFF71A
S31508003460D6FF0028FBD1FFF7D9FF0028FBD1DFF8EC
S31508003470D403DFF8C0130860DFF8CC03DFF8B8130D
S315080034800860DFF8B8130860DFF8C003016831F494
S31508003490FE410160016851F47F010160DFF888038D
S315080034A00168490849000160016851F080710160AE
S315080034B0002010BD10B5040000F05CF920602068FB
S315080034C000F06CF96060606800F073F9A0606068ED
S315080034D000F079F9E06010BD10B50024032824D166
S315080034E0FFF766FFDFF86813401A04D0401E06D0BF
S315080034F0401E0BD011E000F03DF904008DE0FFF707
S3150800350028FF002801D0DFF84C4386E0FFF731FF9B
S31508003510002801D04FF400447FE000F02BF900F0BA
S315080035203DF900F050F9040077E00C2824D1FFF7A4
S315080035303FFFDFF82413401A04D0001F06D0001FEF
S315080035400BD011E000F016F9040066E0FFF701FF62
S31508003550002801D0DFF8FC425FE0FFF70AFF0028E9
S3150800356001D04FF4004458E000F004F900F016F9D1
S3150800357000F01FF9040050E0B0F5406F27D1FFF7BF
S3150800358017FFDFF8D812884207D0DFF8D41288422E
S3150800359007D0B0F10C2F0BD011E000F0EBF80400C7
S315080035A03BE0FFF7D6FE002801D0DFF8A84234E05A
S315080035B0FFF7DFFE002801D04FF400442DE000F0AD
S315080035C0D9F800F0EBF800F0FEF8040025E0302802
S315080035D023D1FFF7EDFEDFF88C12401A04D010381D
S315080035E006D010380BD011E000F0C4F8040014E03F
S315080035F0FFF7AFFE002801D0DFF858420DE0FFF7CD
S31508003600B8FE002801D04FF4004406E000F0B2F8F6
S3150800361000F0C4F800F0CDF80400200010BD10B585
S315080036200024C02824D1FFF7CBFEDFF83C12401A4D
S3150800363004D0403806D040380BD011E000F09AF894
S31508003640040095E0FFF785FE002801D0DFF8044264
S315080036508EE0FFF78EFE002801D04FF4004487E085
S3150800366000F088F800F09AF800F0A3F804007FE06C
S31508003670B0F5407F27D1FFF7A3FEDFF8F0118842A7
S3150800368007D0DFF8EC11884207D0B0F1032F0BD032
S3150800369011E000F06FF804006AE0FFF75AFE002810
S315080036A001D0DFF8B04163E0FFF763FE002801D0E0
S315080036B04FF400445CE000F05DF800F06FF800F0AD
S315080036C078F8040054E0B0F5405F27D1FFF778FE9C
S315080036D0DFF8A011884207D0DFF89C11884207D08E
S315080036E0B0F1302F0BD011E000F044F804003FE0B1
S315080036F0FFF72FFE002801D0DFF8584138E0FFF722
S3150800370038FE002801D04FF4004431E000F032F8CA
S3150800371000F044F800F04DF8040029E0B0F5404FF9
S3150800372026D1FFF74DFEDFF85411884207D0DFF89F
S315080037305011884207D0B0F1C02F0BD011E000F02D
S3150800374019F8040014E0FFF704FE002801D0DFF89A
S3150800375004410DE0FFF70DFE002801D04FF40044A8
S3150800376006E000F007F800F019F800F022F8040067
S31508003770200010BD80B50020FFF702FE002804D007
S31508003780042804D0082804D006E0324805E03D485D
S3150800379003E000F022F800E02E4802BD10B5040050
S315080037A0FFF7F4FD3849C0F30310085CC440200055
S315080037B010BD10B50400FFF7EFFD3449800A085C18
S315080037C0C440200010BD10B50400FFF7EBFD2F49DB
S315080037D0400B085CC440200010BD70B500200020D6
S315080037E0FFF7FDFD002803D0B0F5800F02D003E0F7
S315080037F0184C02E0234C00E0164CFFF702FE0500C9
S31508003800FFF7F3FD0600B4FBF5F006FB00F6FFF73D
S31508003810F2FD000C401C4000B6FBF0F070BD000045
S3150800382000380240703802407438024008380240B6
S3150800383090380240043802408438024088380240F2
S31508003840FFFFF2EA10300024003000240C38024052
S31508003850010003000024F40004000C000004000C1E
S315080038600008000C100030004000C00000010003F2
S31508003870000200030010003000200030004000C0A5
S31508003880008000C000127A00585D0008945D0008A8
S3150800389038B500F02BF9DFF808544021681C00F011
S315080038A03CF92870DFF8FC434021601C00F035F92C
S315080038B020702878FF2802D02078FF2804D1842198
S315080038C0DFF8E403FEF759FEDFF8E0430022DFF8ED
S315080038D0E0132000FEF790FCDFF8D8132000FEF76F
S315080038E0B7FC0120FEF771FE2000FEF7BBFCD4F8FA
S315080038F09802FDF77FFF00F010FAB0F5FA6F03D2D1
S315080039004FF4FA6000F006FA31BD10B5DFF89C43B3
S31508003910D4F89802FDF781FF2000FEF785FC002009
S31508003920FEF753FE10BD70B505000C002000C0B2AE
S31508003930402804DBB921DFF87003FEF71EFE2000DD
S31508003940C0B200F069F8C0B2012804D0BD21DFF882
S315080039505803FEF712FE00260EE0FFF7FBF93000CB
S3150800396080B2285C00F058F8C0B2012803D0C621FE
S31508003970CD48FEF702FE761C30002100C9B280B29F
S3150800398089B28842E9D370BD2DE9F04105000E00E1
S31508003990C648D0F89802FDF7B3FCC74C2078002833
S315080039A013D1C64D280000F02FF801280AD128782F
S315080039B0002807D02878402804DA01202070002043
S315080039C0BF4908700020BDE8F081BD4FDFF8EC82E2
S315080039D038784044401C00F017F80128F2D13878AE
S315080039E0401C3870387898F800108842EAD13A783E
S315080039F092B218F10101280000F0C8F900202070E1
S31508003A00387830700120DEE780B50100A5480078D7
S31508003A1000F0E8F8C0B202BD80B50100C9B2A048FE
S31508003A20007800F091F8C0B202BD7CB59C4C2078B5
S31508003A3000F022F905002800C0B2002827D0280087
S31508003A40C0B2412800DB4025002612E069462078EE
S31508003A5000F0C8F8C0B2012804D04FF4A371924808
S31508003A60FEF78BFD9DF8000096493200D2B28854C5
S31508003A70761C30002900C0B2C9B28842E6D3EDB23E
S31508003A802B009BB28F4A81218848FEF777FB73BDCE
S31508003A90F8B50600002000F004FA0400834D310052
S31508003AA0C9B22800FEF786FB070000260FE03000A3
S31508003AB080B2215C7B48007800F046F8C0B2012845
S31508003AC004D04FF4B4717848FEF757FD761C3000E1
S31508003AD0390080B289B28842E9D300F0E2F90200DF
S31508003AE0402301212800FEF757FBF1BD10B4764BA1
S31508003AF0190013F11802002004E088744A6118318D
S31508003B001832401C0400E4B2002CF6D08874002059
S31508003B1048616E48036010BC704710B46B4B1A6856
S31508003B20002A01D1FF200DE01A6854691C6011743F
S31508003B309060D060002353741060C9B20844401ED8
S31508003B405060907C10BC704738B505000C00280002
S31508003B50C0B2022804DB4FF4E0715348FEF70DFDAE
S31508003B60182059492A00D2B242430A44527C2B00F3
S31508003B70DBB243430B441B7C9A4201D1002030E060
S31508003B802A00D2B242430A44D26814702A00D2B23A
S31508003B9042430A442B00DBB243430B445B7C5B1C69
S31508003BA053742A00D2B242430A442B00DBB2434381
S31508003BB00B44DB685B1CD3602A00D2B242430A443A
S31508003BC052682B00DBB243430B44DB689A4207D2A8
S31508003BD02A00D2B242430A44EDB245434859D0605E
S31508003BE0012032BD38B504000D002000C0B20228FD
S31508003BF004DB4FF4F1712C48FEF7BFFC1821324A5A
S31508003C002000C0B248431044407C002801D100205F
S31508003C1031E02000C0B2484310448068007828701C
S31508003C202000C0B2484310442300DBB24B43134480
S31508003C305B7C5B1E43742000C0B2484310442300DB
S31508003C40DBB24B4313449B685B1C83602000C0B205
S31508003C504843104440682300DBB24B4313449B6837
S31508003C60984207D22000C0B248431044E4B24C43FD
S31508003C7011598160012032BD10B504002000C0B280
S31508003C80022804DB40F202210748FEF776FC0E49BB
S31508003C90E4B21820444301EB0400407C10BD000048
S31508003CA0F80D00203C0E0020E05B0008C40400204C
S31508003CB06C0000201400002017100020C00E002001
S31508003CC016100020000F0020800F0020081000208A
S31508003CD080B501201749087000F022F800F001F8B5
S31508003CE001BD10B500F078F9012812D0114C2078E2
S31508003CF001280ED1FDF7CDF90F490A680F49096861
S31508003D008A1812F5FA72904203D30020207000F048
S31508003D101BF810BD084908607047074800687047D7
S31508003D2080B504480078012803D1FDF7B2F90349A4
S31508003D30086001BD12100020F80F0020F40F0020C3
S31508003D4080B500F053F901BD10B500F05FF9002801
S31508003D5016D0FEF720FC002812D000F0EBF8FDF78D
S31508003D608BF900F070F900F055F906490840064944
S31508003D70086000F04FF9001D046800F039F9A04703
S31508003D8010BD000080FFFF1F08ED00E070B50400BD
S31508003D900D00160005E0287820706D1C641CFEF7DF
S31508003DA0D9FF3000461E80B20028F4D170BD00004D
S31508003DB038B5040000254023022281212000FEF7A1
S31508003DC07DF94023022201212000FEF777F94023DE
S31508003DD0354A01212000FEF7DFF92800C0B232BDBE
S31508003DE038B50400002581212000FEF779F9012164
S31508003DF02000FEF775F92800C0B232BD38B50B00B1
S31508003E0017222A4C14F109011D7815F0600F29D1E3
S31508003E105D78062D04D00A2D14D00B2D17D021E07D
S31508003E205D88ADB22D0AADB2212D07D114F112016C
S31508003E30DA88182A01DB172200E0DA8892B2FEF740
S31508003E404BFF0FE001221A49FEF746FF0AE05988A0
S31508003E50C9B2002903D198781549086002E019000B
S31508003E60FEF7FEFE002032BD80B5FFF7DEFD00201E
S31508003E7002BD80B50800C0B2FFF70AFE002002BDE9
S31508003E8080B590F87402032801D1FFF7CEFD002013
S31508003E9002BD20210180054870470A210180054896
S31508003EA07047014870470000400F00204C00002072
S31508003EB00C1000200800002010B500F0E9F800F00A
S31508003EC035FB434C0120207000F015FC00202070C3
S31508003ED0FFF7DEFC0220207010BD1CB53D4C69467C
S31508003EE0200000F0BBFB012807D1012038490870E3
S31508003EF09DF80010200000F0EBF86946200000F05D
S31508003F0036FC012807D10020314908709DF80010B9
S31508003F10200000F0DDF869462000FFF735FD01288E
S31508003F2007D102202A4908709DF80010200000F0E9
S31508003F30CFF813BD80B5FFF7E8FC01BD70B50400E6
S31508003F400D00234E3078012804D12900C9B220007B
S31508003F5000F055FB3078002804D12900C9B22000AA
S31508003F6000F0E4FB3078022804D12900C9B2200009
S31508003F70FFF7D9FC00F0A6F870BD154800780028B0
S31508003F8005D0022807D004D3032806D007E040202E
S31508003F9006E0082004E03F2002E0002000E0402080
S31508003FA080B270470A480078002805D0022807D052
S31508003FB004D3032806D007E0402006E0082004E0E2
S31508003FC03F2002E0002000E0402080B27047000059
S31508003FD0BC000020800E002010B5002400F069F80F
S31508003FE0002800D001242000C0B210BD72B6704768
S31508003FF062B6704780B500F037FC01BD80B500F0A9
S315080040003CFC02BD80B500F06DFC02BD80B500F039
S31508004010C7FC02BD80B500F004FD02BD80B500F006
S315080040208AFC002801D1002001E000F0E1FC02BD75
S3150800403080B5032000F065FE002000F089FE00F040
S31508004040BBFF002002BD80B50C485FF0FF31016060
S31508004050002202600A4801600022026009480160E5
S3150800406000220260084801600022026007480160D9
S315080040700021016001F012F8002002BD203802403C
S3150800408024380240103802401438024018380240DA
S31508004090DFF8C8030021017000218164002180F83F
S315080040A043100021A0F844100021817000214170BE
S315080040B07047DFF8A8030078002801D1002000E047
S315080040C0012070470020DFF8941381F843007047F9
S315080040D010B50178FF2917D100F08CF8DFF87C437A
S315080040E094F84300012802D1102000F07BF8B4F9B7
S315080040F04400012807DB012084F84300B4F9441082
S31508004100E01C00F053F810BDDFF8501309780129B8
S315080041104BD10178C92932D0CC293FD0CF293AD002
S31508004120D0292FD0D12933D0D2292ED0F32917D090
S31508004130F4290FD0F5290AD0F6290ED0FA2912D07B
S31508004140FC2913D0FD2914D0FE2915D029E000F04A
S31508004150B5F8C3E700F0D1F8C0E700F0A6F8BDE768
S3150800416000F0ECF8BAE700F08EF8B7E700F086F84A
S31508004170B4E700F072F8B1E700F063F8AEE700F0D4
S3150800418004F9ABE700F020F9A8E700F0E9F8A5E79D
S3150800419000F048F9A2E700F057F99FE700F062F946
S315080041A09CE7202000F01EF898E7ACE780B589B2B6
S315080041B0FFF7C4FE01BDF8B504000D001600002780
S315080041C004E02078C719641CFEF7C4FD2800451EC4
S315080041D00028F6D1FFB237600120F2BD00209F49C2
S315080041E0487070479D49FE22CA7008710220A1F8DE
S315080041F04400704710B5FFF7F1FF984C0120207076
S31508004200FF20E07000202071207950F01000207106
S315080042100020607160796071FFF7AFFEA071FFF74B
S31508004220C1FEE071FFF7BEFE80B2000A20720120CF
S3150800423060720120A0720820A4F84400FFF7DAFE95
S3150800424010BD10B5854C00202070FFF7C7FFFF2072
S31508004250E0700120A4F8440010BD8048FF21C17019
S315080042600021017141784171002181710021C171DC
S31508004270002101720621A0F84410704780B500207D
S31508004280FFF7B0FF01BD7548FF21C170744981640D
S315080042900021017100214171002181710721C0F8B7
S315080042A007100821A0F8441070476C49FF22CA700D
S315080042B0406888640120A1F84400704738B50400B6
S315080042C0FFF75BFE80B2401E6178884203DA22203F
S315080042D0FFF788FF10E06278604D281D92B2A96C3E
S315080042E0FFF754FDFF20E870A86C61784018A864B1
S315080042F06078401CA5F8440031BD38B50400FFF7C6
S315080043003CFE80B2401E6178884203DA2220FFF71D
S3150800431069FF12E0514D6068A8646278281D92B260
S31508004320A96CFFF733FDFF20E870A86C6178401888
S31508004330A8646078401CA5F8440031BD10B5474C08
S31508004340FF21E170E21D4168A06CFFF734FF207180
S31508004350002060710020A0710820A4F8440010BD58
S3150800436010B53E4CFF20E0700020207100206071DF
S31508004370FFF703FEA0710020E071002020720020E4
S3150800438060720720A4F8440010BD38B50400FFF792
S31508004390F4FD0100314D621C89B2491EA86CFFF775
S315080043A02DFE002803D13120FFF71CFF0BE0FF206C
S315080043B0E870FFF7E2FDA96C80B2401E4018A864B9
S315080043C00120A5F8440031BD38B50400FFF7D5FD36
S315080043D080B2801E6178884203DA2220FFF702FF46
S315080043E01FE01E4DFF20E8700120A5F84400607804
S315080043F0002807D1FFF712FE002802D13120FFF767
S31508004400F1FE0EE0A21C6178A86CFFF7F7FD002804
S3150800441003D13120FFF7E6FE03E0A86C6178401867
S31508004420A86431BD10B50D4C4168A06CFFF7EAFDD4
S31508004430002803D13120FFF7D5FE04E0FF20E07005
S315080044400120A4F8440010BD80B5FFF77DFC0348A1
S31508004450FF21C1700121A0F8441001BD680D00209C
S31508004460A45D000880B53120FFF7BCFE01BD000041
S31508004470F8B584B004000D0016001F006846FFF763
S3150800448019F802984FF47A71B0FBF1F1002200E0B6
S31508004490521C1000C0B2122845D2864B200080B2AA
S315080044A094465FFA8CFC13F81CC096465FFA8EFE9B
S315080044B003EB4E0E9EF801E01EEB0C0C1CF1010CF2
S315080044C00CFB00F0B1FBF0FC00FB1C100028DFD150
S315080044D0200080B294465FFA8CFC13F81CC09646FE
S315080044E05FFA8EFE03EB4E0E9EF801E01EEB0C0CF7
S315080044F01CF1010C0CFB00F0B1FBF0F028802888B9
S315080045000028C5D0288840F2014C6045C0DA100062
S31508004510C0B213F810003070D2B203EB42004078F4
S315080045203870012000E0002005B0F0BD30B58BB032
S315080045300020ADF8020000208DF8010000208DF85B
S31508004540000040F267656B460DF101020DF10201AC
S315080045504FF4FA70FFF78CFF002803D1B5215648AF
S31508004560FEF70BF8554C56482060002020760020B0
S3150800457060760020A0760120E076002020770020D3
S3150800458060770020A0600020E0609DF80100401ED2
S31508004590000420619DF80000401E00056061BDF81A
S315080045A0020060602000FEF70FFC002D02D46D05A6
S315080045B0444805E025F00045ED0055F0040542485D
S315080045C00021069100210791012108912900090C73
S315080045D00191ADB202950100090C039180B20490D5
S315080045E000200590012009900E200A9001A92000BC
S315080045F0FEF7A0FC2000FEF72FFD0BB030BD30B54E
S3150800460087B0020040F2E170002803D40190002030
S31508004610039004E020F0004002900420039000205C
S315080046200490C9B20591254D6B4601A92800FEF7ED
S3150800463043FDC0B200280FD1FCF72BFD040032342D
S3150800464000992800FEF7BDFD002805D0FEF782FB7D
S31508004650FCF71FFD8442F3D207B030BD78B587B0AA
S3150800466003000C0040F2676600256A4600211348DD
S31508004670FEF7BDFD002812D1002E07D40098B042DF
S315080046800DD1029800280AD1012508E026F0004637
S315080046900198B04203D10298042800D101252800C8
S315080046A0C0B2012801D1049820702800C0B208B011
S315080046B070BD00007C5C0008A45B0008B00F0020F9
S315080046C0006400400400E0FFFCFF1F00016851F091
S315080046D0010101607047C069400910F00100704788
S315080046E0C069C00910F001007047406AC0B270473F
S315080046F0C9B28162704718B587B04FF4614000901F
S315080047000020019000200290002003900C200490C5
S3150800471000200590002006904D4C6946200000F0C8
S315080047203CFD2000FFF7D2FF08B010BD70B50400AD
S315080047300D002800C0B2412803DB81214548FDF75A
S315080047401CFF2800C0B200F06BF8002607E0FEF751
S3150800475001FB300080B2205C00F062F8761C300065
S315080047602900C9B280B289B28842F0D370BD2DE95A
S31508004770F04105000E00384C2078002815D1374D39
S31508004780280000F03DF8012837D12878002834D0D1
S315080047902878412831DAFCF77CFC3149086000208A
S315080047A0304908700120207027E02E4FDFF8AC80D2
S315080047B038784044401C00F023F8012814D1387892
S315080047C0401C3870387898F80010884215D13A7825
S315080047D092B218F101012800FFF7D8FA00202070DC
S315080047E038783070012009E0FCF753FC1C49096849
S315080047F06431814201D2002020700020BDE8F0819A
S3150800480038B50400124D2800FFF765FF002805D0CB
S315080048102800FFF76AFF2070012000E0002032BD63
S3150800482038B501000A4DC9B22800FFF761FFFCF749
S3150800483030FC04000A342800FFF752FF002805D18F
S31508004840FEF788FAFCF725FC8442F4D231BD000055
S3150800485000480040645B000815100020B40D0020D5
S3150800486000100020141000205FF0FF30DFF8D4138A
S315080048700860DFF8D41308607047F8B504000D0027
S315080048801600DFF8C873B96CF86C4118491E091B85
S31508004890681E814201D2002023E0200000F0A9F919
S315080048A0FF2805D02819401E00F0A3F9FF2801D1DA
S315080048B0002016E02100490A4FF400704143386889
S315080048C0814207D12B0032002100DFF87C0300F07B
S315080048D0DCF806E02B0032002100DFF8680300F060
S315080048E0D4F8F2BD70B504000D00DFF86003816CE2
S315080048F0C06C4118491E091B681E814201D200205E
S3150800490018E0200000F075F906002C19641E200036
S3150800491000F06FF93100C9B2FF2903D00100C9B20E
S31508004920FF2901D1002005E00100C9B23000C0B25C
S3150800493000F01EF970BD80B500200090C2490868D5
S3150800494010F1010F01D1012029E0009A4868821868
S315080049500092009A886882180092009AC86882189D
S315080049600092009A086982180092009A486982188B
S315080049700092009A886982180092009AC86982187B
S3150800498000920098C04300900098401C00906A4628
S315080049900421AE48006810F5E470FFF76EFF02BD0B
S315080049A00021AA4A1068006841181068001D0068AE
S315080049B04118106808300068411810680C30006803
S315080049C041181068103000684118106814300068E3
S315080049D041181068183000684118106810F5E4701E
S315080049E000684118002901D1012000E00020704725
S315080049F080B59548016811F1010F05D000F08FF8D0
S31508004A00002801D100200BE08E48016811F1010F42
S31508004A1005D000F084F8002801D1002000E001202C
S31508004A2002BD8A480068704780B5CA0501D00020D3
S31508004A300BE002688A4201D1012006E001604FF4CA
S31508004A400072001DFFF7A2F9012002BD38B5040067
S31508004A500D007D48844208D17A4C29002000FFF7D2
S31508004A60E3FF00280FD100200EE078490A68954236
S31508004A7002D104000D68F0E7200000F050F8002885
S31508004A80EBD1002000E0200032BD2DE9F041040002
S31508004A90884616001D0047467F0A4FF400704743B4
S31508004AA0206810F1010F07D139002000FFF7BCFF7D
S31508004AB0002801D100202EE02068B84208D039002D
S31508004AC02000FFF7C3FF0400002C01D1002022E0DC
S31508004AD02068B8EB000804EB080010F10408FEF79C
S31508004AE039F9201DB8EB0000B0F5007F09D317F59A
S31508004AF000712000FFF7AAFF0400002C0DD014F166
S31508004B000408307888F8000018F10108761C6D1E34
S31508004B10002DE4D10120BDE8F0810020FBE72DE956
S31508004B20F0410500012600F001FC002704E0D8F852
S31508004B300000A04215D17F1C802F13D2D5F8008023
S31508004B4018EB870805EB87004468FEF703F922008F
S31508004B5000234146022000F0A3FB0028E7D00026E8
S31508004B6000E0002600F0F2FB3000C0B2BDE8F0819C
S31508004B7078B585B004000D000126002000902800B5
S31508004B802100C0B2C9B2884200D200262F482100AF
S31508004B90027AC9B2914205D390F850002900C9B2E9
S31508004BA0884200D200263000C0B201281DD100205C
S31508004BB00190022004900120039000F0B7FB00E06A
S31508004BC0641C28002100C0B2C9B288420BD3FEF784
S31508004BD0C1F82000C0B20290694601A800F064FC42
S31508004BE00028EDD0002600F0B1FB3000C0B206B0B8
S31508004BF070BD70B50400FF25002600E0761C300065
S31508004C00C0B207281AD2FEF7A5F80C210F4A3000C1
S31508004C10C0B2484310588442F0D33000C0B248436B
S31508004C2013583000C0B2484310444068C3189C4229
S31508004C30E4D2F6B24E4302EB0600057A2800C0B26B
S31508004C4070BD00006007002064090020BC5A0008F7
S31508004C5010F00700374B1A684FF6FF010A4036492D
S31508004C6051EA00210A431A60704732480068C0F3C7
S31508004C7002207047020052B2002A04D409012F4AC2
S31508004C8040B2115407E009012D4A40B210F00F0056
S31508004C90104400F8041C704710B410F00700D0F157
S31508004CA00703052B01D3042301E0D0F10703041DF4
S31508004CB0072C01D2002000E0C01E012414FA03F3D9
S31508004CC05B1E1940814014FA00F0401E104008434C
S31508004CD010BC704780B5411EB1F1807F01D3012019
S31508004CE00EE0401E174908600F215FF0FF30FFF7FE
S31508004CF0C1FF0020144908600720144908600020F5
S31508004D0002BD80B5FFF7A4FF01BD70B504000D0014
S31508004D1016000020FFF7A9FF32002900FFF7BCFFA5
S31508004D200100200040B2FFF7A5FF70BD80B5FFF770
S31508004D30D1FF02BD0CED00E00000FA0500E400E03A
S31508004D4018ED00E014E000E018E000E010E000E0F4
S31508004D5010B504004FF47A700D490978B0FBF1F0EC
S31508004D600C490968B1FBF0F0FFF7E0FF002801D015
S31508004D7001200CE0102C09D2002221005FF0FF3040
S31508004D80FFF7C3FF04480460002000E0012010BDBF
S31508004D90BD0000200400002000000020D94801685A
S31508004DA051F4803101607047D6490A6832F44042AE
S31508004DB0104308607047D448016851F480210160A7
S31508004DC07047D148016851F4803101607047CE4878
S31508004DD00068400C10F001007047CC490A68920838
S31508004DE09200104308607047C848006810F00C002D
S31508004DF07047C6490A6832F0F002104308607047E7
S31508004E00C2490A6832F4E052104308607047BF4945
S31508004E100A6832F46042104308607047BA4801686D
S31508004E2051F0807101607047B7480068400E10F075
S31508004E300100704770B4B64D2E68B64C2640304314
S31508004E40084350EA82101843286070BC704770B453
S31508004E50AF4D2E68B04C26403043084350EA8210C6
S31508004E601843286070BC704781B0AC490A68024391
S31508004E700A60096808400090009801B07047A74981
S31508004E800A6832EA00000860704781B0A4490A68D7
S31508004E9002430A60096808400090009801B070470C
S31508004EA09F490A6832EA00000860704781B09D4948
S31508004EB00A6802430A60096808400090009801B031
S31508004EC0704798490A6832EA00000860704781B05E
S31508004ED095490A6802430A600968084000900098E4
S31508004EE001B0704790490A6832EA000008607047C6
S31508004EF08E490A68120912011043086070478B48E8
S31508004F00006810F00F00704709048161704780B58A
S31508004F1000F005F800F05CFB00F068FBFCE780B5E4
S31508004F20FFF786F800F001F801BD80B50720FFF706
S31508004F30DFFFFFF7E4FF072803D067217C48FDF76A
S31508004F401CFB4FF44040FFF72FFFFFF727FFFFF743
S31508004F5032FFFFF736FFFFF73AFF0128FBD10023A0
S31508004F604FF4D87208215FF48000FFF763FF5FF003
S31508004F7010634FF4D87208215FF48000FFF767FFCB
S31508004F80FFF74CFFFFF750FF0128FBD10020FFF782
S31508004F9030FF4FF4A050FFF733FF4FF40040FFF700
S31508004FA036FF0220FFF719FFFFF71EFF0828FBD17F
S31508004FB0604800F025FB01BD38B586B04FF4804047
S31508004FC0FFF785FF5FF08050FFF770FF0120FFF7BE
S31508004FD04BFF0220FFF748FF0420FFF745FF082094
S31508004FE0FFF742FF5FF48020FFF760FF5FF0007075
S31508004FF0FFF75CFF802000900120019000200290BE
S3150800500000200390002004904B4C6946200000F0D5
S3150800501011FC80212000FFF777FF4FF40050009025
S3150800502000200190002004906946444800F002FCE4
S315080050304FF440750095022001900320029000204D
S315080050400390002004900720059069463C4800F02C
S31508005050F1FB0095022001900320029000200390A6
S3150800506000200490092005906946200000F0E2FB24
S315080050704FF4C050009002200190032002900020B7
S315080050800390002004900A20059069462D4800F0F8
S31508005090D1FB8020FFF7F9FE07B030BD10B5FEF74B
S315080050A0C4F9254C80212000FFF72EFF244800F084
S315080050B02FFB224800F02CFB200000F029FB21489A
S315080050C000F026FB8020FFF7EBFE5FF00070FFF78D
S315080050D0F8FE5FF48020FFF7F4FE0820FFF7CFFE06
S315080050E00420FFF7CCFE0220FFF7C9FE0120FFF7D8
S315080050F0C6FE5FF08050FFF7E4FE4FF48040FFF7EE
S31508005100F1FE10BD00700040003802400838024029
S31508005110043802400080BCFF0080BFF030380240EF
S31508005120343802404038024044380240003C0240CD
S31508005130105B000800E6DF0C00040240000802408D
S31508005140000C024000000240006810F001007047A1
S31508005150426832F44052114341607047826832F423
S315080051604072114381607047B2F5004F0ED11A00A4
S31508005170520812EB4102B2FBF3F189B24FF6F07214
S315080051800A40C1F342010A43C26005E011EB53012C
S31508005190B1FBF3F189B2C1607047F8B505000F009D
S315080051A0012600242800FFF7CFFF002862D12968CE
S315080051B03A48014078680143F86801433869014371
S315080051C0B86901432960B9682800FFF7C1FF796902
S315080051D02800FFF7C3FF2948854204D10320FEF7BC
S315080051E07BF904003AE02648854204D10C20FEF7F4
S315080051F073F9040032E02348854204D13020FEF7D3
S315080052006BF904002AE02048854204D1C020FEF745
S3150800521006FA040022E01D48854205D14FF4407085
S31508005220FEF7FDF9040019E01948854205D14FF447
S315080052304060FEF751F9040010E01648854205D192
S315080052404FF44050FEF7EBF9040007E01248854298
S3150800525004D14FF44040FEF7E2F90400002C09D0CF
S315080052603868002806D000263B68BA69210028005D
S31508005270FFF77AFF3000C0B2F2BD0000001001400F
S315080052800044004000480040004C004000500040E8
S315080052900014014000780040007C0040F369FFEFED
S315080052A02DE9F84381460E0014001D000120DFF8A1
S315080052B0E071387D012801D1022035E001203875DA
S315080052C04CF25038404600F048F80100C9B20029AF
S315080052D027D1300022002B00B9F1000F07D0B9F111
S315080052E0020F0ED008D3B9F1030F0ED010E011004B
S315080052F0C9B200F091F80BE0110089B200F07BF812
S3150800530006E0110000F066F802E000F04EF8FFE74C
S31508005310404600F022F8DFF87C110A68520852006D
S315080053200A6000213975C0B2BDE8F28300205949E8
S315080053300A68002A08D5594A594B1360594B136015
S315080053400968002900D50120C0B270475148016894
S3150800535051F0004101600020704738B50400002074
S3150800536000204B498861FBF7A5FE05004A480168FD
S31508005370C9030BD514F1010FF8D0002C04D0FBF7A4
S3150800538099FE401B8442F1D203200DE0016811F01A
S31508005390F20F03D000F04FF8012005E00168C907B5
S315080053A001D501210160002032BD10B439490C68CD
S315080053B034F440740C600C6854F440740C600C6847
S315080053C054F001040C600260001D0360BFF34F8FA8
S315080053D010BC70472F4A136833F440731360136880
S315080053E053F400731360136853F0010313600160EC
S315080053F0BFF34F8F7047274A136833F4407313601F
S31508005400136853F480731360136853F00103136031
S315080054100180BFF34F8F70471E4A136833F44073F9
S31508005420136013681360136853F001031360017067
S31508005430BFF34F8F704718480168890704D5144988
S315080054408A6952F020028A610168C90604D51049A2
S315080054508A6952F010028A610168890604D50C49E6
S315080054608A6952F008028A610168490604D5084922
S315080054708A6952F004028A610168090604D504495A
S315080054808A6952F002028A61F221016070470000BF
S31508005490D80F0020103C02400C3C0240043C02405D
S315080054A023016745AB89EFCD2DE9F04104000D00D6
S315080054B001200020DFF81061307D012801D102208B
S315080054C03EE0012030754CF250373800FFF745FFB3
S315080054D00100C9B2002930D15FF0FF312960216887
S315080054E001290DD1E068C0B200F02CF83800FFF7AA
S315080054F034FFDFF8D8100A6832F004020A601CE0AC
S31508005500D4F8048001E018F10108A26861688A18D5
S31508005510904512D2E168C9B2404600F026F8380034
S31508005520FFF71BFF29490A6832F07A020A60010070
S31508005530C9B20029E7D0C5F8008000213175C0B28C
S31508005540BDE8F08121490A6832F440720A600A68A7
S3150800555052F004020A600A68C0B2000250F48030B1
S3150800556010430860BFF34F8F704700220A00D2B27B
S31508005570002A01D100210EE00A00D2B2012A02D186
S315080055804FF4807107E0C9B2022902D14FF40071C5
S3150800559001E04FF440710D4A136833F44073136009
S315080055A0136819431160116831F0F8011160116828
S315080055B0C00050F0020008431060106850F48030B4
S315080055C01060BFF34F8F7047D80F0020103C024081
S315080055D080B5FEF7B5FBFDF7B9FBFBF73DFDFEF71A
S315080055E009FDFEF769FCFEF773FB01BD80B5FDF703
S315080055F0B1FBFBF745FDFEF770FCFEF772FB01BD3C
S3150800560001490860704700000400002030B40468AF
S3150800561091FAA1F3B3FA83F30325DBB25B009D404D
S31508005620AC4391FAA1F1B1FA81F1C9B249008A40B5
S315080056302243026030BC704743688B435143194389
S315080056404160704730B4846891FAA1F3B3FA83F3E2
S315080056500325DBB25B009D40AC4391FAA1F1B1FA98
S3150800566081F1C9B249008A402243826030BC704742
S3150800567030B4C46891FAA1F3B3FA83F30325DBB215
S315080056805B009D40AC4391FAA1F1B1FA81F1C9B230
S3150800569049008A402243C26030BC704730B4046A6D
S315080056A091FAA1F3B3FA83F30F25DBB29B009D4071
S315080056B0AC4391FAA1F1B1FA81F1C9B289008A40E5
S315080056C02243026230BC704730B4446A0B001B0A9E
S315080056D093FAA3F3B3FA83F30F25DBB29B009D403D
S315080056E0AC43090A91FAA1F1B1FA81F1C9B289006C
S315080056F08A402243426230BC704742490A681043D6
S31508005700086070473F490A6832EA00000860704737
S3150800571010B500243C49884206D10120FFF7EDFF69
S315080057200120FFF7EFFF6AE03849884206D10220D8
S31508005730FFF7E3FF0220FFF7E5FF60E03449884200
S3150800574006D10420FFF7D9FF0420FFF7DBFF56E058
S315080057503049884206D10820FFF7CFFF0820FFF717
S31508005760D1FF4CE02C49884206D11020FFF7C5FF2F
S315080057701020FFF7C7FF42E02849884206D12020BB
S31508005780FFF7BBFF2020FFF7BDFF38E0244988421A
S3150800579006D14020FFF7B1FF4020FFF7B3FF2EE008
S315080057A02049884206D18020FFF7A7FF8020FFF70F
S315080057B0A9FF24E01C49884208D14FF48070FFF7FE
S315080057C09CFF4FF48070FFF79DFF18E01749884249
S315080057D008D14FF40070FFF790FF4FF40070FFF701
S315080057E091FF0CE01249884208D14FF48060FFF718
S315080057F084FF4FF48060FFF785FF00E00124200056
S31508005800C0B210BD10380240000002400004024039
S3150800581000080240000C024000100240001402403A
S3150800582000180240001C02400020024000240240EA
S3150800583000280240F8B505000E0000200020306858
S3150800584090FAA0F0B0FA80F72FE0726921002800DC
S31508005850FFF73AFF28E034680120B8400440002CDE
S3150800586022D0726821002800FFF7D0FE7068012850
S3150800587002D07068022804D1B26821002800FFF718
S31508005880E1FE326921002800FFF7F2FE706802285F
S315080058900AD194FAA4F0B0FA80F00828D5D2726931
S315080058A021002800FFF7FAFE7F1C3068F840002820
S315080058B0D1D17068012802D07068022804D1F26834
S315080058C031682800FFF7B8FE0020F2BD12200880D4
S315080058D02D487047042008802C48704780B50A0078
S315080058E0C0B2002804D12A492A48FDF7C4F903E0C2
S315080058F027492848FDF7BFF9254802BD10B50A0013
S31508005900234C21002448FDF7B6F9200010BD80B5C8
S315080059101A20088000F022F8204802BD80B50A0047
S31508005920C0B2002804D11A491D48FDF7A4F903E0BE
S3150800593017491B48FDF79FF9154802BD80B50A00AF
S31508005940C0B2002804D112491648FDF794F903E0BD
S315080059500F491448FDF78FF90D4802BD38B51248AE
S31508005960006812490C6812490968081800280AD004
S315080059700A4D0822A91C00F01DF8042215F112018F
S31508005980200000F017F831BD880000209C00002098
S31508005990680B0020445D0008685D0008A000002030
S315080059A09C5D00082C5D000820F4F01F24F4F01F0D
S315080059B028F4F01F30B4002300231AE00400240F53
S315080059C037341D00EDB201F815400AE00400240F33
S315080059D00A2CF3D20400240F30341D00EDB201F86E
S315080059E01540000100241D00EDB201EB45056C7061
S315080059F05B1C1C001500E4B2EDB2AC42E6D330BC29
S31508005A00704700000F48016851F4700101600E49A3
S31508005A10086850F00100086000200C4A10600A6807
S31508005A200B4802400A600B480B4A1060086830F4BD
S31508005A30802008600020094908605FF00060084976
S31508005A400860704788ED00E00038024008380240D8
S31508005A50FFFFF6FE10300024043802400C380240DE
S31508005A6008ED00E0433A5C576F726B5C736F6674BF
S31508005A70776172655C4F70656E424C545C54617216
S31508005A806765745C44656D6F5C41524D434D375F85
S31508005A9053544D333246375F4E75636C656F5F46B8
S31508005AA03734365A475F4941525C426F6F745C75AA
S31508005AB07362645F636F6E662E6300000080000881
S31508005AC000800000010000000000010800800000BE
S31508005AD002000000008001080080000003000000AA
S31508005AE0000002080000020004000000000004088C
S31508005AF0000004000500000000000808000004007B
S31508005B000600000000000C08000004000700000062
S31508005B10433A5C576F726B5C736F66747761726534
S31508005B205C4F70656E424C545C5461726765745C78
S31508005B3044656D6F5C41524D434D375F53544D3349
S31508005B403246375F4E75636C656F5F463734365A33
S31508005B50475F4941525C426F6F745C6D61696E2E96
S31508005B6063000000433A5C576F726B5C736F667430
S31508005B70776172655C4F70656E424C545C54617215
S31508005B806765745C536F757263655C41524D434D2E
S31508005B90375F53544D333246375C72733233322E85
S31508005BA063000000433A5C576F726B5C736F6674F0
S31508005BB0776172655C4F70656E424C545C546172D5
S31508005BC06765745C536F757263655C41524D434DEE
S31508005BD0375F53544D333246375C63616E2E63002C
S31508005BE0433A5C576F726B5C736F66747761726564
S31508005BF05C4F70656E424C545C5461726765745CA8
S31508005C00536F757263655C41524D434D375F53540C
S31508005C104D333246375C7573622E630030B50168C2
S31508005C2084684218416802EB5103C90703D54C44FE
S31508005C3001E0491C05D19A420AD012F9011B12F853
S31508005C40015B002904F8015BF3D4491EF7D5F2E796
S31508005C500C3030BD10B5074979441831064C7C44E0
S31508005C60163404E00A68081D114488470146A14213
S31508005C70F8D110BD500000006C00000005020602B5
S31508005C80060307030803090309040A040B040C04A2
S31508005C900C050D050E050F050F0610061007100852
S31508005CA04EF68851CEF20001086840F4700008608C
S31508005CB0BFF34F8FBFF36F8F4FF00070E1EE100AFE
S31508005CC070470000FBB3FFFF5C0F0000C000002018
S31508005CD00000000049FFFFFF7802000030010000C5
S31508005CE00000002000F00DF8002801D0FFF7B2FFF1
S31508005CF0AFF300800020AFF30080FFF708F900F04B
S31508005D0002F80120704700F001B80000074638463F
S31508005D1000F002F8FBE7000080B5AFF30080024A06
S31508005D2011001820ABBEFBE72600020057696E5526
S31508005D3053422042756C6B20496E746572666163C6
S31508005D406500000057696E5553422042756C6B20FA
S31508005D5044657669636500000000000000000000E5
S31508005D6001020304060708094F70656E424C542069
S31508005D7055736572000000000148804701480047D6
S31508005D80055A0008895D0008AFF30080FFF788FF11
S31508005D90FFF7A8FF000000000102030444656661DE
S31508005DA0756C74004F70656E424C5400FFF7FEBF69
S31508005DB0FFF7FEBFFFF7FEBFFFF7FEBFFFF7FEBF09
S31508005DC0FFF7FEBFFFF7FEBFFFF7FEBFFFF7FEBFF9
S31508005DD0FFF7FEBFFFF7FEBFFFF7FEBFFFF7FEBFE9
S31508005DE0FFF7FEBFFFF7FEBFFFF7FEBFFFF7FEBFD9
S31508005DF0FFF7FEBFFFF7FEBFFFF7FEBFFFF7FEBFC9
S31508005E00FFF7FEBFFFF7FEBFFFF7FEBFFFF7FEBFB8
S31508005E10FFF7FEBFFFF7FEBFFFF7FEBFFFF7FEBFA8
S31508005E20FFF7FEBFFFF7FEBFFFF7FEBFFFF7FEBF98
S31508005E30FFF7FEBFFFF7FEBFFFF7FEBFFFF7FEBF88
S31508005E40FFF7FEBFFFF7FEBFFFF7FEBFFFF7FEBF78
S31508005E50FFF7FEBFFFF7FEBFFFF7FEBFFFF7FEBF68
S31508005E60FFF7FEBFFFF7FEBFFFF7FEBFFFF7FEBF58
S31508005E70FFF7FEBFFFF7FEBFFFF7FEBFFFF7FEBF48
S31508005E80FFF7FEBFFFF7FEBFFFF7FEBFFFF7FEBF38
S31508005E90FFF7FEBFFFF7FEBFFFF7FEBFFFF7FEBF28
S31508005EA0FFF7FEBFFFF7FEBFFFF7FEBFFFF7FEBF18
S31508005EB0FFF7FEBFFFF7FEBFFFF7FEBFFFF7FEBF08
S31508005EC0FFF7FEBFFFF7FEBFFFF7FEBFFFF7FEBFF8
S31508005ED0FFF7FEBFFFF7FEBFFFF7FEBFFFF7FEBFE8
S31508005EE0FFF7FEBFFFF7FEBFFFF7FEBFFFF7FEBFD8
S31508005EF0FFF7FEBFFFF7FEBFFFF7FEBFFFF7FEBFC8
S31508005F00FFF7FEBFFFF7FEBFFFF7FEBFFFF7FEBFB7
S31508005F10FFF7FEBFFFF7FEBFFFF7FEBFFFF7FEBFA7
S31508005F20FFF7FEBFFFF7FEBFFFF7FEBFFFF7FEBF97
S31508005F30FFF7FEBFFFF7FEBFFFF7FEBFFFF7FEBF87
S31508005F40FFF7FEBFFFF7FEBFFFF7FEBFFFF7FEBF77
S31508005F500010FC000624F4000A060002FD000140B9
S31508005F6001FD000BB13D0008E13D0008FD3D0008BC
S31508005F70F8000B693E0008733E0008813E0008F4ED
S31508005F800003933E0008FC00129B3E00080902200D
S31508005F9000010100C0320904000002FFFD002D07C0
S31508005FA00581024000FF070501024000FFCD5800A9
S31508005FB008D5580008FD580008DD5800080F590094
S31508005FC0081D5900083D59000812010002FD00127B
S31508005FD040501DAC600002010203010000040309E1
S30D08005FE0041A03E6000104019E
S70508005D890C
